:100000000C9444010C9461010C947C010C946101EA
:100010000C9461010C9461010C9461010C946101D8
:100020000C9461010C9461010C9476170C9461019D
:100030000C9461010C9461010C9461010C946101B8
:100040000C9461010C9461010C9461010C946101A8
:100050000C94610195059505C105C105290659074F
:10006000590759074706E006F106F10629001E0068
:100070001F002000210022002D0035002E0023004B
:1000800024002500260027002A002B0014001A0057
:100090000800150017002F00310030001C00180068
:1000A0000C00120013003400390004001600070091
:1000B00009000A004A004C004B000B000D000E0026
:1000C0000F0033002800E1001D001B00060019008E
:1000D00005004D0052004E001100100036003700A0
:1000E0003800E500E000E300E20001512C002C00A4
:1000F000500051004F002C002C000151E600E70099
:10010000E4003A003B003C003D003E003F0053004D
:1001100038002502400041004200430044004500F1
:10012000AF00B200B300B100C75CC65C5F00600006
:1001300061002D0001000100460047004800AC00AE
:10014000AE00AB00AD00C95CC85C5C005D005E0049
:100150002E020100005C010001000100AA00A800BD
:10016000A9006500CB5CCA5C59005A005B005800CE
:100170000100010001000100010001000100C35C59
:100180000151C55CC45C6200010063005800580066
:10019000015101000100010009023B00020100A021
:1001A000FA09040000010301010009210101000115
:1001B0002240000705810308000109040100010332
:1001C000000000092101010001223200070583031C
:1001D0000800011201100100000008EDDE0100011D
:1001E00000010200010E03700075006E006B003705
:1001F00000350000001A036400730061006E0063A4
:1002000000680065007A007300650063006F0000FD
:10021000000403090405010980A101850319012ACD
:10022000B700150126B700950175108100C0050CB7
:100230000901A101850419012AA002150126A002C5
:10024000950175108100C005010906A10105071976
:10025000E029E715002501950875018102950175D2
:100260000881030507190029FF150026FF009506E0
:100270007508810005081901290595057501910288
:10028000950175039103C00011241FBECFE5D8E08E
:10029000DEBFCDBF10E0A0E6B0E0E4E5F6E302C0CB
:1002A00005900D92AC3FB107D9F722E0ACEFB0E07A
:1002B00001C01D92A23BB207E1F70E9440130C94CB
:1002C000281B0C940000A82FB92F80E090E041E09B
:1002D00050EA609530E009C02D9182279795879567
:1002E00010F084279527305EC8F36F5FA8F3089558
:1002F000EADF8D939D930895CF93CFB7CF93DF938C
:10030000C395839BE9F7839B10C0839B0EC0839B9F
:100310000CC0839B0AC0839B08C0839B06C0C0910E
:100320008902C395C09389028EC06F93C0918802E1
:10033000DD27C057DD4F2F9365E5839B03C02F91C9
:100340006F91E1CF0F931F934F9320E040E15F93B4
:1003500000B30C7003FB27F93F9350E03BE039C03A
:100360001C7040642F77012F5F5F1EC0406810B380
:100370001C702F7752501FC0406400B32F770C7051
:10038000D1F15F5F00C023C0406210B32F771C70B3
:1003900091F15F5F00C025C00C701027515012F41E
:1003A0005D5F0000115027952C3F10B3C8F61C70FC
:1003B0000127015027952C3FC8F64227499300B3E7
:1003C0000C7010274F73115027952C3FA8F64695B7
:1003D000469510B31C7079F00127015027952C3FEA
:1003E00098F66B5A60F3315000B3B0F600C010E8D5
:1003F0001ABF00271CC03B503195C31BD04010E8EA
:100400001ABF0881033C21F10B3411F120918502C0
:100410001981110F1213EDCF4A81441F093679F16A
:100420000D3211F0013E29F74F7009F0042F0093AF
:100430008E023F915F914F911F910F912F916F917C
:10044000CAB7C7FD5DCFDF91CF91CFBFCF911895D0
:1004500020918E02222369F310918C02112309F05E
:1004600049C034300AF448C030938C02209387028C
:10047000109188023BE0311B309388023DC000910F
:100480008C020130BCF50AE54F7049F430917100DF
:1004900034FD33C000937100C2E6D2E032C0433075
:1004A00059F0443091F030916D0234FD26C0009334
:1004B0006D02CEE6D2E025C03091A60234FD1DC00B
:1004C0000093A602C7EAD2E01CC03091790234FD45
:1004D00014C000937902CAE7D2E013C0052710E0E8
:1004E00000C0000002BB1AC0052710E0221F1DC07B
:1004F00010E021C04AE502C032ED432FC4E1D0E054
:1005000032E011B31C60939A02B311BB5CE020E8A7
:1005100065E320FF052702BB279517951C3FF0F6E2
:100520006695B8F7B1F720FF052702BB2795179509
:100530001C3FD0F62795179517FF052700001C3F95
:1005400002BBB0F629913A9519F7037F10918D02FD
:10055000110FC651D04002BB11F01093850210E874
:100560001ABF086011B3137F402F437F54E05A95A0
:10057000F1F702BB11BB42BB5CCFD09A0C94F711D0
:10058000CF93C82F0E94BD03882329F0C1FD02C06C
:10059000D89A01C0D898CF910895FA019281E82F96
:1005A000E295EF70282F2F70F0E032A9992341F0E7
:1005B00081E090E001C0880F2A95EAF7832B08C0FC
:1005C00081E090E001C0880F2A95EAF780958323A7
:1005D00082AB0895AB01BC0180E90E94CD0281E0AD
:1005E0000895823038F4662311F089EA01C08AEA5E
:1005F0000E94430581E0089581E008950C94EA0289
:1006000008950C9400031F93CF93DF9300D000D084
:100610001F92CDB7DEB749835A836B833091FF00B9
:1006200089819A81311114C0662359F0222349F03F
:100630000E949209182F682F89819A810E943B0994
:1006400003C00E946609182F69817A81812F04C036
:100650000E94920969817A810F900F900F900F90FC
:100660000F90DF91CF911F910C94CA10FC01262F9F
:10067000408151816281738184810C94030381E004
:100680000895CF93DF93EC0160E00E943603BE0132
:10069000DF91CF910C9401030C94BD020C94F511E1
:1006A00008950E94E5070E9450032FEF84E39CE029
:1006B000215080409040E1F700C000000C949C174E
:1006C0000F931F93CF93DF938C0161E00E94360359
:1006D000EC01B8010E94FE028823F1F1B801CE01BD
:1006E0000E9431168823C1F1B801CE010E944D133A
:1006F000882391F1B801CE010E948D15882361F104
:10070000F8018281882309F1CB358DE5D807C1F046
:1007100050F4C115FCE5DF0781F0CF3DDC45A9F4BD
:100720000E94C30E19C0CC35EDE5DE0761F0CD3572
:10073000DD4559F40E940C0E08C00E9451030CC004
:100740000E94150E02C00E94180EC801DF91CF91C1
:100750001F910F910C94FC0280E0DF91CF911F91CB
:100760000F9108950E9420170C94C9030E94CC0396
:100770000C94261708950C94BA0381E00895089507
:10078000CF93C82F0E94BB038C2F0E94C002CF9131
:10079000089580E00C94C0030E948D160C94C00351
:1007A0000E948D169091FE00891721F08093FE0023
:1007B0000C94C0030895CF93DF93CDB7DEB72B978A
:1007C0000FB6F894DEBF0FBECDBF4F835887698741
:1007D0007A878B8761110E94580D9E012F5F3F4FD2
:1007E00086E0F90111928A95E9F785E0FE013796D6
:1007F000D90101900D928A95E1F789819A814C8106
:100800005D81452B31F09F3F31F491E08F3F19F42A
:1008100003C091E001C090E090FF09C049815A8176
:100820006B817C818D819E810E94790C05C0C901FC
:100830000E943F038111F2CF2B960FB6F894DEBFD2
:100840000FBECDBFDF91CF910895FC0180819181D2
:100850000E94D4090895CF93882309F49CC0C82F1F
:100860008238C1F40E948D1681FD95C069E38091A4
:100870006200909163000E9412170E947A0D2FEF80
:1008800081EE94E0215080409040E1F700C00000EC
:1008900069E319C0833801F50E948D1680FD7BC085
:1008A00063E580916200909163000E9412170E949C
:1008B0007A0D2FEF81EE94E0215080409040E1F7D7
:1008C00000C0000063E580916200909163000E9487
:1008D0001417CF910C947A0D8438C1F40E948D16B0
:1008E00082FD59C067E480916200909163000E948C
:1008F00012170E947A0D2FEF81EE94E02150804074
:100900009040E1F700C0000067E4DDCF8CEF8C0F72
:10091000813AD0F46C2F80916200909163000E9424
:10092000DC16882349F06C2F80916200909163005F
:100930000E9414170E947A0D6C2F80916200909192
:1009400063000E941217C5CF80E28C0F883048F4F4
:10095000C77081E001C0880FCA95EAF70E943B0D7D
:10096000B8CFEBE5EC0FE33040F4F0E0E056FF4F9A
:10097000808190E0CF910C94A416C85AC73158F4E6
:10098000EC2FF0E0EE0FFF1FEE58FF4F80819181BA
:10099000CF910C94BA16CF910895882309F45BC0C7
:1009A000682F823879F40E948D1681FF54C069E364
:1009B00080916200909163000E9412170E947A0D4C
:1009C00069E310C08338B1F40E948D1680FF43C0E4
:1009D00063E580916200909163000E9412170E946B
:1009E0007A0D63E580916200909163000E94141774
:1009F0000C947A0D843879F40E948D1682FF2BC0F6
:100A000067E480916200909163000E9412170E9437
:100A10007A0D67E4E7CF8CEF860F813A18F380E216
:100A2000860F883048F4677081E001C0880F6A95AE
:100A3000EAF70E94410DDCCF8BE5860F833020F46E
:100A400080E090E00C94A416685A673120F480E0AE
:100A500090E00C94BA1608951F93CF93DF93182F4C
:100A6000EB010E942B04209741F08FE99FE0019752
:100A7000F1F700C000002197F6CF812FDF91CF91D1
:100A80001F910C94CD04893319F06AE070E002C024
:100A900060E570E00C942C05882321F00E943B0D4A
:100AA0000C947A0D0895882321F00E94410D0C9436
:100AB0007A0D0895CF92DF92EF92FF920F931F93DA
:100AC000CF93DF937C01D62FC72FFC0112810581C4
:100AD00002950F700E94310D8823B9F01123A9F0FF
:100AE0008C2F807F803421F080E28D0F883068F079
:100AF0008091490282FD09C082E00E94DA0D0E94C5
:100B0000310D91E0D82ED92601C0D12CCC2EC29423
:100B10008FE0C8228C2D90E08C30910508F0C9C17F
:100B2000FC01E65DFF4F0C94C01A8C2F807FCF70C4
:100B3000882311F0C295C07F112399F0CC2309F4CA
:100B40009FC180E28D0F883010F0D11104C08C2F2E
:100B50000E943B0D03C08C2F0E944B0D0E947A0D0A
:100B60008FC18D2F0E94CD04CC2309F4A2C180E255
:100B70008D0F883038F1DD2329F18C2F0E94510D23
:100B800024C08C2F807FCF70803211F0C295C07F3F
:100B9000DD2319F0D130A1F13DC08091490282FFDF
:100BA00017C0112349F0CC2329F08C2F0E943B0D54
:100BB0000E947A0D80E065C180E00E94CD04CC23C4
:100BC00009F477C18C2F0E94410D0E947A0D71C1EA
:100BD000112371F0002341F0013031F40E945B0DCC
:100BE0008C2B0E94630D65C10E945B0D8C2B1DC078
:100BF000002319F0013009F45CC10E94700D25C07A
:100C0000112321F0063008F054C10EC0053008F061
:100C100050C11BC0112361F0002331F0F701858121
:100C200080FF2EC18F7085838C2F0E944C0541C19F
:100C3000002359F0D93309F033C1FFEF07EE13E079
:100C4000F15000401040E1F72FC18C2F0E94530556
:100C500030C18C2F86958695837019F0813061F0B4
:100C600028C1112321F08D2F9C2F937002C080E0AA
:100C700090E00E94A41625C1112321F08D2F9C2FF6
:100C8000937002C080E090E00E94BA161AC18C2FC7
:100C9000837009F047C0111110C12D2F22952695A0
:100CA0002770220F220F6D2F6F70862F90E0A0E02B
:100CB000B0E0022E04C0880F991FAA1FBB1F0A9420
:100CC000D2F7D4FF10C04FE050E060E070E004C005
:100CD000440F551F661F771F2A95D2F740955095F0
:100CE0006095709503C040E050E0BA01C695C69586
:100CF000C3708A019B01082B192B2A2B3B2BC9019E
:100D0000B801C23049F058F4C13019F00E945108BE
:100D1000D4C00E943F08D1C00E946308CEC00E9488
:100D20003D08CBC0112319F08C2F817001C086952E
:100D3000882309F4C2C02D2F229526952770220FF3
:100D4000220F6D2F6F70862F90E0A0E0B0E0022E92
:100D500004C0880F991FAA1FBB1F0A94D2F7D4FFA3
:100D600010C04FE050E060E070E004C0440F551F39
:100D7000661F771F2A95D2F740955095609570951C
:100D800003C040E050E0BA01C695C695C3708A0121
:100D90009B01082B192B2A2B3B2BC901B801C23010
:100DA00049F058F4C13019F00E94160986C00E941B
:100DB000040983C00E94280980C00E9477087DC072
:100DC000CF70112339F08C2F0E949D088D2F0E9427
:100DD0004C0573C08D2F0E9453058C2F0E94BE08B6
:100DE0006CC0D23F21F128F4D03F41F0D13FC1F097
:100DF00043C0D33F19F1D43F79F03EC0112341F0F5
:100E0000053008F056C08C2F8F710E94E30851C046
:100E1000063008F04EC0F7CF8091490282FF18C01B
:100E2000112339F08C2F8F710E949D0842C011232D
:100E3000C9F38C2F8F710E94BE083BC0112329F08B
:100E40008C2F8F710E94880834C00E94830831C0A3
:100E5000112349F0CF718C2F0E949D0863E08C2FE5
:100E60000E94BF0D26C081E00E94DA0D023008F119
:100E700082E00E94DA0D1DC0112331F0002391F2AF
:100E80008D2F0E942B0415C0002399F2D93341F411
:100E90001FEF27EE33E0115020403040E1F704C04F
:100EA0008FE39CE90197F1F700C000008D2F0E94AD
:100EB000CD0488EF8C0D843020F40E948D160E94A2
:100EC000C003DD20C9F00E942D0D80FD15C0F70183
:100ED00012820E94270D0E949D08C7010E949D0753
:100EE0000E94270DDF91CF911F910F91FF90EF90FE
:100EF000DF90CF900C94BE08DF91CF911F910F919E
:100F0000FF90EF90DF90CF9008950F931F93CF93B2
:100F1000DF93EC01688179818A810E94DF098C016D
:100F20000E943A090E942B08B801CE010E945A057E
:100F3000DF91CF911F910F910895CF93DF93EC0133
:100F4000988189812B813C81232B31F08F3F31F4B3
:100F500081E09F3F19F403C081E001C080E080FD83
:100F60001DC0CE010E946003811110C00E94310D8E
:100F70008823A1F08A81882389F08091490282FD2B
:100F80000DC082E0DF91CF910C94DA0DCE010E946A
:100F90008507CE01DF91CF910C944103DF91CF9172
:100FA000089580E090E00E94A41680E090E00E9406
:100FB000BA160E94580D0C947A0D8091620090919F
:100FC00063000E9416170C94D1070E94480D0C94E0
:100FD000DD0792959F70963079F010F4925001C021
:100FE0009A50923068F4803F69F018F4883E40F4DB
:100FF00009C0843F29F406C0883E20F0813F11F0EB
:1010000080E0089581E00895FC01808191810E9433
:10101000D4090E94E9070895CF93DF9300D000D050
:101020001F92CDB7DEB70F900F900F900F900F90DB
:10103000DF91CF910895CF93DF9300D000D000D0FF
:10104000CDB7DEB726960FB6F894DEBF0FBECDBF84
:10105000DF91CF910895089508950C942C080C9475
:101060002D080E942F0860933601709337018093FA
:101070003801909339010C94D1070C9431080F93E7
:101080001F93009136011091370120913801309162
:101090003901602B712B822B932B1F910F910C9494
:1010A00031080F931F930091360110913701209161
:1010B00038013091390160237123822393231F91DA
:1010C0000F910C9431080F931F93009136011091EA
:1010D000370120913801309139016027712782272B
:1010E00093271F910F910C9431080C942C080E94A7
:1010F00075086093320170933301809334019093AB
:1011000035010C94D10760E070E0CB010C947708B6
:101110000F931F9341E050E060E070E08A019B0173
:1011200004C0000F111F221F331F8A95D2F7C90177
:10113000B8011F910F910C9477080F931F9341E012
:1011400050E060E070E004C0440F551F661F771F39
:101150008A95D2F78091320190913301A0913401A8
:10116000B09135018A019B01082B192B2A2B3B2BAF
:10117000C901B8011F910F910C9477080F931F9329
:1011800041E050E060E070E004C0440F551F661F6E
:10119000771F8A95D2F7409550956095709580910C
:1011A000320190913301A0913401B09135018A014F
:1011B0009B01082319232A233B23C901B8011F914E
:1011C0000F910C9477080F931F9341E050E060E07B
:1011D00070E004C0440F551F661F771F8A95D2F731
:1011E0008091320190913301A0913401B091350189
:1011F0008A019B01082719272A273B27C901B80123
:101200001F910F910C9477080F931F930091320157
:10121000109133012091340130913501602B712BF5
:10122000822B932B1F910F910C9477080F931F9390
:101230000091320110913301209134013091350138
:1012400060237123822393231F910F910C947708BD
:101250000F931F93009132011091330120913401BB
:101260003091350160277127822793271F910F91B5
:101270000C94770808952FE0929F800D1124E82F99
:10128000E695E695E695877051E001C0550F8A9581
:10129000EAF785E0E89FF0011124E050FF4F20E0DD
:1012A00030E070E04081CB01022E02C09695879518
:1012B0000A94E2F78170819584278523842781939E
:1012C0002F5F3F4F2530310569F708952FE0929F3A
:1012D000800D1124682F669566956695982F9770F6
:1012E00085E0689FB001112440E050E080E0FB0100
:1012F000E40FF51FE050FF4F208130E0092E02C0BF
:10130000369527950A94E2F721703327042E01C001
:10131000220F0A94EAF7822B4F5F5F4F4530510549
:1013200031F70895BF92CF92DF92EF92FF920F9321
:101330001F93CF93DF938C01C0903201D090330183
:10134000E0903401F09035018091360190913701A1
:10135000A0913801B0913901C82AD92AEA2AFB2A7A
:10136000CFE1D0E0D701C6010C2E04C0B695A795F9
:10137000979587950A94D2F780FD04C0219790F73E
:10138000B12C07C0BC2EB8018C2F0E94DD10019734
:10139000A9F38B2DDF91CF911F910F91FF90EF90CB
:1013A000DF90CF90BF900895CF93DF93EC010E9420
:1013B0009209BE010E94DD10DF91CF9108951F9325
:1013C000CF93DF93EB019091FF00992321F0CB01A4
:1013D0000E94D40913C0882349F0CB010E949209CE
:1013E000182F682FCE010E943B0904C0CB010E9438
:1013F0006609182FBE01812F0E94DD10DF91CF9169
:101400001F9108951F93CF93DF93C0913A0116E087
:1014100080913B01C81799F0D0E01C9FF0011D9FFF
:10142000F00D1124E45CFE4F408151816281738193
:10143000848195810E941B082196C770E9CFDF91B6
:10144000CF911F91089540916C0150916D01609171
:101450006E0170916F0180917001909171010C94F7
:101460001B08EF92FF920F931F93CF93DF9380910E
:10147000710182958F7009F065C080916E0188239B
:1014800009F460C080913A01F0903B0110916C0129
:1014900000916D0160916F017091700191E01F3FAB
:1014A00009F090E0C0916000D0916100292F96E092
:1014B000E92E8F1509F446C06115710521F00F3F23
:1014C00021F030E003C031E001C0322F90E030FD68
:1014D00036C0E89EF001E99EF00D1124DF01A45C06
:1014E000BE4F11963C911197301329C03C91311396
:1014F00026C012963C911297311121C013964D913E
:101500005C911497461B570B4C175D07C0F48091F4
:1015100071018F70806180937101EF5BFE4F80815C
:101520008F70806180838CE691E00E949D07DF913F
:10153000CF911F910F91FF90EF900C94020A0196AA
:101540008770B7CFDF91CF911F910F91FF90EF90F0
:1015500008959F92AF92BF92CF92DF92EF92FF9247
:101560000F931F93CF93DF93CDB7DEB761970FB67D
:10157000F894DEBF0FBECDBF8C0185E0F801DE011F
:101580001D9601900D928A95E1F7D8011296EC9084
:1015900090916C01E0916D0120916F01309170018B
:1015A0002115310531F0EF3F31F481E09F3F19F40F
:1015B00003C081E001C080E0B82FB1709B2E80FD98
:1015C00047C1D8014C9111965C9111971396AD903B
:1015D000BC9014978CE6C82E81E0D82EF0906E0156
:1015E000B501621B730B2091600030916100FF20F8
:1015F00009F4D9C0809171016217730708F095C092
:10160000282F207F09F052C05E1313C0491311C068
:10161000FE2CE1100EC08F708061809371010E94DA
:10162000230AC6010E949D0780917101F8018583FC
:101630004DC1AB2831F05F3F31F481E04F3F19F4E9
:1016400003C081E001C080E080FD03C081E08E2501
:1016500002C080E090E0F82FF170FF2E80FF1CC0E8
:1016600080913A0120913B0136E0821709F40BC1C9
:1016700090E0389FF001399FF00D1124E45CFE4F9B
:101680006181561306C06081461303C06281E61271
:1016900003C001968770E9CFFE2CEE2009F416C135
:1016A0008091710181608093710154C05E1306C006
:1016B000491304C0E11002C0F80199C0C8010E949A
:1016C0000408882361F1EE2051F120917101822FED
:1016D00082958F7090E0029774F080916C019091E8
:1016E0006D0198878F831986BB86AA862C87CE01C9
:1016F00007960E949D0786E0F801ACE6B1E00190F4
:101700000D928A95E1F70E94310A0E94230A0AC0CD
:101710005E1711F1C8010E94040881112CC0C80194
:101720000E949D07FF24F394D1C0282F207F81F7CA
:101730007A2DB98AA88A6E2D89890E940C088CE6B8
:1017400091E00E949D0786E0D6011D928A95E9F7F7
:101750000E94230AF12CBAC04913DCCFE110DACF82
:10176000F8018583C8010E949D0786E0D6011D927D
:101770008A95E9F7ABC0EE2091F220917101822F9A
:1017800082958F7090E002970CF4B5CF80916C0138
:1017900090916D019A8389831B82BD82AC822E83D6
:1017A000CE010196A6CF6217730708F044C0FE2C45
:1017B000EE2009F4B4CF5E1330C049132EC020913F
:1017C000710120FD21C0822F82958F70482F50E03B
:1017D00041155105C9F0F80125834F30510541F0FD
:1017E0008F5F982F9295907F822F8F70892B8583A2
:1017F000C8010E949D0786E0F801ACE6B1E00190C7
:101800000D928A95E1F73CC086E0F801ACE6B1E0C4
:1018100001900D928A95E1F759C0C8010E94040811
:10182000811169CF80917101816080937101C8013C
:101830000E949D074BC07A2DB98AA88A6E2D89898E
:101840000E940C0886E0D6011D928A95E9F718C01F
:10185000EE2009F464CFC8010E940408F82E882302
:1018600009F45DCF86E0F801ACE6B1E001900D929D
:101870008A95E1F78CE691E00E9425040E94310AE6
:101880000E94230A23C04D875E878D859E850E9416
:10189000D409292F22952F70223028F49F7039F017
:1018A000811105C00BC0243028F49F7049F4805E7C
:1018B000883020F0C8010E949D079F2CF92C06C09B
:1018C000D80115969C91907F91F7F8CF8F2D619656
:1018D0000FB6F894DEBF0FBECDBFDF91CF911F9141
:1018E0000F91FF90EF90DF90CF90BF90AF909F90BF
:1018F00008951F93CF93DF93CDB7DEB72C970FB624
:10190000F894DEBF0FBECDBF4F83588769877A87B3
:101910008B879C87CE0107960E94A90A8823D1F065
:101920009F8188852A853B85232B31F08F3F31F4B9
:1019300081E09F3F19F403C081E001C080E080FD99
:1019400047C04F81588569857A858B859C850E9423
:101950001B083EC086E0FE013796DE01119601901D
:101960000D928A95E1F7FF81E8856A857B8561158F
:10197000710531F0EF3F31F481E0FF3F19F403C00E
:1019800081E001C080E080FD23C020913B0130E078
:10199000C90101968770992740913A0150E0841758
:1019A0009507F1F1F983EA837D836C8396E0929F3A
:1019B000D001939FB00D1124A45CBE4FFE0131965F
:1019C00001900D929A95E1F780933B010E94020AE3
:1019D00016E080913A0190913B01891771F1189FAF
:1019E000C0011124845C9E4F0E94A90A882329F11A
:1019F000E0913A011E9FF0011124E45CFE4F40810A
:101A0000518162817381848195810E941B0880913C
:101A10003A0190E001968770992780933A01D9CFD7
:101A20000E94E50710923B0110923A01ECE6F1E0CA
:101A300086E0DF011D928A95E9F72C960FB6F8949F
:101A4000DEBF0FBECDBFDF91CF911F910895809172
:101A50007A01859585958595089580917A0187709D
:101A6000089590917A01977081E009F480E00895DB
:101A700080918501089590918501892B809385013E
:101A8000089580959091850189238093850108951B
:101A900010928501089590918401892B809384018F
:101AA00008958095909184018923809384010895FD
:101AB00010928401089580917B01089508950C94FB
:101AC0005E0D0C945F0D9091490292FD08C09091BB
:101AD0007B01981721F080937B010C94610D089590
:101AE00080917B01882329F010927B0180E00C9487
:101AF000610D0895CF93DF93E0916200F091630050
:101B0000809185018083E0916200F0916300908173
:101B100080918401892B808380917B01882381F0CF
:101B2000E0916200F09163009081892B8083809125
:101B30006200909163000E94D01681110E94700D86
:101B4000C0916200D091630048E050E062E771E02C
:101B5000CE010E94DA1A892B69F088E0FE01A2E723
:101B6000B1E001900D928A95E1F7CE01DF91CF911E
:101B70000C949916DF91CF9108950C945E0D90917D
:101B8000490292FD10C098E0899F90011124262BF4
:101B900020937A010E949D0880917A018595859510
:101BA00085950C94BD0D0C949D0810927A0180E0EF
:101BB0000C94BD0D20917A018095822380937A0147
:101BC000982F977099F430E0482F082E000C550B91
:101BD0002417350759F09091490292FD07C0859569
:101BE000859585950E94BE080C94D50D0895909119
:101BF000490292FB222720F9281769F080FB92F90D
:101C00009093490280914802909149020E943F0EB0
:101C100082E00C94DA0D08958091490282FB8827B6
:101C200080F991E089270C94F70D81E00C94F70D71
:101C300080E00C94F70D80E090E00E94EF1A21E024
:101C4000893E9E4F09F020E0822F089582E090E0C7
:101C50000C94E71A83E090E00C94E71ACF9384E0A9
:101C600090E00E94E71AC82F82E290E00E94E71AF3
:101C70002C2F30E0A901582BCA01CF910895CF93A2
:101C8000C92F682F84E090E00E94F51A6C2F82E241
:101C900090E0CF910C94F51AAB01BC018FE090E07D
:101CA0000C94061BAB01BC0183E190E00C94061B75
:101CB00060E070E0CB010C94520E60E070E0CB016C
:101CC0000E944C0E0C94580E69EE7EEF80E090E07E
:101CD0000E94121B60E082E090E00E94F51A60E032
:101CE00083E090E00E94F51A1092360110923701BD
:101CF000109238011092390160E084E090E00E9477
:101D0000F51A60E082E290E00E94F51A60E085E05A
:101D100090E00E94F51A60E086E090E00E94F51ADB
:101D20006FEF87E090E00E94F51A40E050E0BA01C2
:101D300088E090E00E94061B60E08DE090E00E9449
:101D4000F51A40E050E0BA0188E190E00E94061BDD
:101D500060E087E190E00E94F51A40E050E0BA01AF
:101D60008CE190E00E94061B60E070E080E290E071
:101D70000E94121B40E050E0BA0188E190E00E940E
:101D8000061B0C945D0E0C94640E682F8EE090E0A0
:101D90000C94F51A0E945B17609398017093990157
:101DA00080939A0190939B016093940170939501A5
:101DB000809396019093970108950E945B1760931A
:101DC00098017093990180939A0190939B0160937D
:101DD00090017093910180939201909393010895E3
:101DE00084B7806884BF84B7806884BF089581E029
:101DF00008950C94F70E08950C94FB0E0C94FB0EB2
:101E00000C94FE0E0C94FB0E0C94020F0C94FB0E23
:101E10000E94F00E89EB91E10E9483160E94060F4A
:101E20000C94040F0E94FC0E0C94FB0E0E94BC113B
:101E30000C94BF030E9448170E949F120E94160F25
:101E40000E949E140C94000F5F926F927F928F926B
:101E50009F92AF92BF92CF92DF92EF92FF920F9339
:101E60001F93CF93DF93CDB7DEB72A970FB6F894C1
:101E7000DEBF0FBECDBF0E94B412C82E81110E94DA
:101E8000CA0E36E8832E31E0932E00E010E0502E8B
:101E9000802F0E94E0115C01F401619071904F016C
:101EA0006826792661147104B1F40F5F1F4F053065
:101EB000110569F78FEF89838A831B820E944F1770
:101EC0008160782F9D838C8349815A816B818D81BC
:101ED0000E94DB033AC080919C0181FD0E94E911C0
:101EE000D12CEE24E394F12CC3018E219F21892B68
:101EF00029F10E94F90E8823A9F0DE825F82AE20CC
:101F0000BF2081E0AB2809F480E088870E944F174A
:101F10008160782F9A8789874E815F8168858A855D
:101F20000E94DB03000F111FF801EA57FE4F80816A
:101F30009181E826F926F182E08207C0D394EE0C65
:101F4000FF1CFFE0DF12D0CFB0CF81E0C11001C095
:101F500080E02A960FB6F894DEBF0FBECDBFDF91AA
:101F6000CF911F910F91FF90EF90DF90CF90BF9096
:101F7000AF909F908F907F906F905F9008950E9498
:101F8000240F0E94F01481110E94DD0E0C94D003E6
:101F9000CF93DF930E94E210EC01811522E59207B6
:101FA000E8F5811531E5930708F0B6C0883E910544
:101FB00028F5803E910508F0E9C0883A910570F453
:101FC000853A910508F07AC08130910509F473C013
:101FD00008F4D9C0049708F0D9C0D5C08F3B91054B
:101FE00008F0D1C0C85AD0E0CC0FDD1FCD55DF4F6F
:101FF0000990D881C02DCE019464C9C0811540E5F7
:10200000940708F069C0811550E4950708F060C096
:102010009A9581159F4108F4B9C0B5C0811536E580
:10202000930728F5811545E5940708F092C08115BE
:1020300054E5950708F087C0AC0143705527282F59
:1020400026952695C115D34508F06CC081E090E037
:1020500002C0880F991F4A95E2F740E2249F900141
:102060001124EC01C22BD32BCE019C6890C08115AA
:102070002AE5920780F4811539E5930708F072C0CC
:10208000811548E5940708F47EC0D82FCC27CE01EF
:10209000806F906A7CC090568115904208F073C0A2
:1020A0008D2F8F710E947611DD27D0628F71AE0166
:1020B000582BCA016CC081E090E069C0C55AD0E0DD
:1020C000CF52DF4F8881C82FD0E0CE0190645FC02F
:1020D000DF70CE01906A5BC074E0969587957A9523
:1020E000E1F7282F23703C2F337081E090E002C08D
:1020F000880F991F3A95E2F79C68AC01522B9A0120
:102100009C2F9F709695969550E2959FE001112423
:10211000C9018C2B9D2B3BC0D82FCC27CE01816FC2
:10212000906A35C081E090E002C0880F991F4A95FF
:10213000E2F750E2259F90011124EC01C22BD32B32
:10214000CE019A6824C0D82FCC27CE01846F906A24
:102150001EC00E9476118F7190E0D82FCC27CE013F
:10216000906215C08F700E94761194E0D695C79545
:102170009A95E1F7CF70D0E0DC2FCC27D0699E0193
:10218000282BC90104C080E090E001C0CE01DF919E
:10219000CF9108952BE4829FC0011124FC012FE010
:1021A000729FE00DF11D1124E60FF11DEE0FFF1FD0
:1021B000E459FF4F8591949108950E94CA100E949E
:1021C000C80F08958238910569F1B0F48133910503
:1021D00009F46DC048F48932910509F463C08A326C
:1021E000910509F469C008958533910509F455C036
:1021F00089339105B9F00895833E910569F138F46A
:10220000803E9105B1F0823E910509F10895863E28
:102210009105A9F1873E9105B9F1843E910509F038
:1022200064C023C02091480220FD4FC021FD4DC055
:1022300008958091480280FD44C08091490280FF4A
:1022400044C08091480284FD42C083EE4DC080911D
:10225000480282FF38C0F5CF8091480282FD33C02A
:102260008091490280FD31C0ECCF8091490281FF0D
:1022700032C08091480284FD2AC087EE35C080912B
:10228000480283FF26C0F5CF8091480283FD21C01C
:102290008091490281FD1FC0ECCF8091480285FDED
:1022A0001CC01DC08091480285FD19C016C08091D8
:1022B000480286FD16C017C08091480286FD13C0F3
:1022C00010C089E311C082EE0FC080EE0DC080E027
:1022D0000BC086EE09C084EE07C089E205C085E325
:1022E00003C08AE201C081E390E008959091480222
:1022F00092FF0DC0282F2871283019F4877F846041
:1023000006C0282F2471243011F48B7F886093FF3E
:102310000DC0282F2871283119F4877E846106C0EA
:10232000282F2471243111F48B7E88612091490279
:1023300020FF0DC0382F3871383019F4877F816045
:1023400006C0382F3171313011F48E7F886021FF43
:102350000DC0282F2871283119F4877E816106C0AD
:10236000282F2171213111F48E7E886194FD877EA2
:10237000089580E0089508950E941B0E811102C007
:102380000E94C30E0E94260E80939C010E942E0E76
:1023900090934902809348020E94BB110E942A0E2A
:1023A000682F70E080E090E00E943D08609132016B
:1023B0007091330180913401909135010C9475082E
:1023C000E82FF0E0EE0FFF1FEC5AFD4F8081918166
:1023D0000895089580EA8A95F1F7089500C0089558
:1023E0000C94EA1108950C94F2110C94F3110C94CE
:1023F000F211F894E82FE295EF70F0E031A9282F60
:102400002F7081E090E001C0880F2A95EAF7982F9D
:102410009095932391AB92A9892B82AB78940895E0
:102420000F931F93CF93DF93C3EED0E089918F3F3B
:1024300011F00E94F91180E0C83ED807B9F7C4ED49
:10244000D0E003EE10E089918F3F11F00E94F91166
:102450000C171D07C1F7DF91CF911F910F910895C0
:10246000BF92CF92DF92EF92FF920F931F93CF9381
:10247000DF938C01C62FD0E0CE018D519F4F6C01B0
:10248000FC0190819F3F09F450C0B62EF894E92FCB
:10249000E295EF70F0E081A99F7021E030E001C08B
:1024A000220F9A95EAF7822B81AB82A920952823E7
:1024B00022AB78940E94EE11E4EDF0E043EE50E0A0
:1024C00021E030E0E12CF12C61916F3F89F0A62FE3
:1024D000A295AF70B0E0D0968C9190E06F7002C082
:1024E000959587956A95E2F780FD02C0C90102C003
:1024F00080E090E0E82AF92A220F331F4E175F0789
:1025000019F7F60180818F3F11F00E94F91161E007
:10251000E114F10409F460E08B2D0E94F011CC0F5E
:10252000DD1FC00FD11FF982E882DF91CF911F918B
:102530000F91FF90EF90DF90CF90BF9008950E9491
:1025400010128AE0E4E5F2E0DF01982F1D929A95DF
:10255000E9F7EAE4F2E0DF011D928A95E9F785E008
:102560000E94FF120C944C03FF920F931F93CF9382
:10257000DF93CDB7DEB72A970FB6F894DEBF0FBE54
:10258000CDBF8E010F5F1F4F8AE0F80111928A952F
:10259000E9F7F12C6F2DC8010E943012F394F5E099
:1025A000FF12F8CF4AE050E0B8018AE492E00E94BE
:1025B000DA1AFF24F394009709F4F12C892B41F0E7
:1025C0008AE0F801AAE4B2E001900D928A95E1F761
:1025D0002F2D45E064E572E08AE492E00E9400134A
:1025E0000E944E038F2D2A960FB6F894DEBF0FBEC1
:1025F000CDBFDF91CF911F910F91FF900895089566
:10260000FF920F931F93CF93DF93F82E092F162F6E
:10261000D72FC42F222349F081E080939F010E948D
:102620004F1790939E0180939D0180919F01882375
:10263000D9F080919D0190919E010E9467170597A6
:1026400098F0EF2DF02FA12FBD2F80E090E04C2FC0
:1026500050E08417950734F4219131912D933D93E7
:102660000196F7CF10929F01DF91CF911F910F91AB
:10267000FF9008950E94B6170E941A0F0C94C71776
:102680000E943D170E94AF170E94080F0E943A1344
:102690000E94D5170E94120FFBCFCF93DF93EC015E
:1026A000FB018281882309F43CC1C430FDE5DF07CA
:1026B00060F4CB3F9CE5D90788F49E0122503C454D
:1026C0002431310508F02EC109C0C236EDE5DE0720
:1026D00029F0C63AFDE5DF0709F024C10E942E0E5D
:1026E0009093490280934802C1318CE5D80709F4E0
:1026F000C6C008F042C0C930ECE5DE0709F49BC053
:1027000000F5C5308CE5D80709F485C078F4C330EE
:10271000ECE5DE0709F478C008F07AC0C230DC4589
:1027200009F0F5C0809148028160EFC0C7309CE598
:10273000D90709F478C008F07AC080914802806116
:10274000E4C0CD30FCE5DF0709F487C058F4CB3096
:102750009CE5D90709F479C008F07BC08091480254
:1027600088606FC0CF30FCE5DF0709F480C008F057
:1027700082C080914802877FC8C0CE3F9CE5D907C0
:1027800009F471C000F5C531FCE5DF0709F485C027
:1027900068F4C3319CE5D90709F475C008F095C009
:1027A0000E94E507809148028F77AFC0CC3FFCE5DF
:1027B000DF07A9F108F054C0CB3FDC4509F0A7C002
:1027C0008091490240C0C230EDE5DE0709F489C0BE
:1027D00058F4C1158DE5D80709F45AC008F069C04E
:1027E0008091490282602FC0C236EDE5DE0709F410
:1027F0007CC0C63AFDE5DF0709F481C0C330DD4582
:1028000009F085C080E06EC08091480282607DC082
:102810008091480216C080914802886076C08091FD
:10282000490282604FC08091480280626EC08091F0
:10283000480280646AC00E94E5078091480280686F
:1028400064C0846062C081603DC0809148028E7F18
:102850005CC0809148028D7F58C08091480216C0AC
:102860008091490218C0809149028D7F2BC08091D0
:1028700048028F7E4AC0809148028F7D46C0809179
:1028800048028F7B42C080914802877F8B7F3DC08A
:10289000809149028D7F8E7F15C08091480282FB16
:1028A000222720F991E0922790FB82F990FB83F98F
:1028B0002CC080914902982F909591708E7F892B22
:1028C00090FB81F98093490222C00E94E507809124
:1028D000480287FB222720F991E0922790FB87F995
:1028E00014C081E00E94C50E12C08091480284FB92
:1028F000222720F991E0922790FB84F906C080916D
:102900004802982F909590FB80F98093480280911F
:102910004802909149020E943F0E0E94E50780E024
:1029200001C081E0DF91CF9108958FE891E0019798
:10293000F1F700C0000008950C94F102CF93DF93EB
:10294000AAEFB0E0C8EFD0E021E030E070E0AC3FAB
:10295000B70759F18D91E82FE295EF70F0E041A9AA
:102960008F70B90102C0660F771F8A95E2F7CB011D
:10297000962F9095942391AB92A9892B82AB899144
:10298000E82FE295EF70F0E041A98F70B90102C025
:10299000660F771F8A95E2F7CB01962F90959423C7
:1029A00091AB92A9892B82ABD1CF0E94951480B3B1
:1029B000982F9170819902C080E001C082E0892B3C
:1029C0008093A40186B386958170B09902C090E08F
:1029D00001C092E0892B8093A501DF91CF910895EA
:1029E0004F925F926F927F928F929F92AF92BF921F
:1029F000CF92DF92EF92FF920F931F93CF93DF93CB
:102A000004EA11E08AEFC82E80E0D82E98EFE92E74
:102A100090E0F92E22EA822E21E0922EC0EAD1E047
:102A20005801512C412C34E0632E712CD501ED91CD
:102A30005D014E2F440F440FF60121916F01E22FEB
:102A4000E295EF70F0E080A990E02F7002C09595BC
:102A500087952A95E2F781709927D7015D917D01CD
:102A6000E52FE295EF70F0E020A930E05F7002C042
:102A7000359527955A95E2F7F901E170FF2720FF78
:102A800002C0E2E0F0E0E82BF92BE42BD801ED9353
:102A90008D01EF70F0E0E851FF4F9081F4018081EB
:102AA000890F808384304CF088818F5F888360E059
:102AB000852D0E949C1421E001C020E0D4018C915E
:102AC0008D3F44F488818150888361E0852D0E9488
:102AD0009C1421E0F4018081082E000C990BB301B5
:102AE0000E94AC1AD4018D934D01422A5394219631
:102AF000B2E05B129BCF842DDF91CF911F910F919C
:102B0000FF90EF90DF90CF90BF90AF909F908F900D
:102B10007F906F905F904F900895CF93DF938631B1
:102B20009C4541F5EB010E94380D982F8A81209138
:102B3000620030916300882379F09A7A81E009F489
:102B400080E08093A601911102C069E201C065E3B3
:102B5000C9010E9412170AC08091A601811102C00A
:102B600069E201C065E3C9010E9414170E947A0D51
:102B700080E001C081E0DF91CF9108950F931F9312
:102B8000CF93DF93C42FD22FFC0182818823C9F019
:102B90004093A9010E944F179093A8018093A70129
:102BA00080E28C0F883008F057C0C77081E001C008
:102BB000880FCA95EAF7DF91CF911F910F910C947E
:102BC0004C058091A901481330C08091A7019091D4
:102BD000A8010E946717883C910538F510E21D0F87
:102BE000CD17B9F080E28C0F883040F4C77081E0D7
:102BF00001C0880FCA95EAF70E945305183028F5DE
:102C000081E09D2F977001C0880F9A95EAF70E9486
:102C10004C05802F0E9443051830F0F4D77081E0F6
:102C200001C0880FDA95EAF70AC080E28C0F88307D
:102C300098F4C77081E001C0880FCA95EAF7DF9168
:102C4000CF911F910F910C945305802FDF91CF915D
:102C50001F910F910C944305DF91CF911F910F911C
:102C600008950F939C01CB01243F4CE5340731F1CB
:102C700088F4293DFCE53F07D9F02A3D4CE53407AF
:102C800079F1283D3C45A9F506E221EE41EE68EDDB
:102C90007CE52BC0263FFCE53F07E1F0A8F0273F8D
:102CA0003C4539F507E225EE46EE67EF7CE51DC0B1
:102CB00007E225EE45EE69ED7CE517C006E221EE60
:102CC00040EE64EF7CE511C007E225EE44EE65EFCF
:102CD0007CE50BC006E221EE42EE66EF7CE505C026
:102CE00008E221E045EE6AED7CE50E94BE1580E039
:102CF00008C0FC018281882319F01092A90101C04B
:102D000081E00F9108959093FD008093FC00089559
:102D10009093AF018093AE010895E091AE01F091E0
:102D2000AF01309721F00190F081E02D099480E00F
:102D30000895E091AE01F091AF01309721F002804B
:102D4000F381E02D099408952091AC013091AD01FB
:102D50002817390771F09093AD018093AC01E09191
:102D6000AE01F091AF01309721F00680F781E02DA0
:102D7000099408952091AA013091AB0128173907D1
:102D800071F09093AB018093AA01E091AE01F091B4
:102D9000AF01309721F00084F185E02D099408956A
:102DA000FC01329697E080E0915029F02191222396
:102DB000D9F38F5FF9CF0895662349F0FC0132966D
:102DC00008962191621729F0E817F907D1F780E0FA
:102DD000089581E008959C01FC0132969FEF80E008
:102DE0004191461789F09F3F19F4411101C0982F76
:102DF0008F5F8630A9F79F3F39F0F901E90FF11D88
:102E000097FDFA956283089508959C012A5F3F4FCC
:102E1000FC014281461301C012820196821793077A
:102E2000B9F708950C94EB160C940517029626E05A
:102E3000FC0111922A95E9F7089508950C941D1745
:102E40000C941E170C941D170C941D170C941D1731
:102E5000CF930E9424170E94B4120E942217C0E050
:102E60008C2F0E94E011892B29F4CF5FC530C1F768
:102E700080E001C081E0CF91089508958091B20172
:102E800081110C94B20308950E94E5070C94B603D7
:102E90008BE083BF8AEF8CBF82E089BF08952FB794
:102EA000F89480915E0290915F02A0916002B091CF
:102EB00061022FBF08952FB7F89460915E02709160
:102EC0005F0280916002909161022FBF08959C0182
:102ED0004FB7F89480915E0290915F02A0916002DA
:102EE000B09161024FBF821B930B089578941F929B
:102EF0000F920FB60F9211248F939F93AF93BF93AE
:102F000080915E0290915F02A0916002B091610297
:102F10000196A11DB11D80935E0290935F02A09364
:102F20006002B0936102BF91AF919F918F910F901A
:102F30000FBE0F901F90189598E088E10FB6F89497
:102F4000A89581BD0FBE91BDA895F894D8E0CEE5B7
:102F500028E3299320E0299314BEFFCF08950E940F
:102F60004F179093B1018093B00108950E94911A78
:102F70008B9A80E0815041F0A895EFE9FFE031970E
:102F8000F1F700C00000F6CF8B98789408950E9466
:102F9000B4180E9488162FEF80E792E021508040FD
:102FA0009040E1F700C000000895809189028823D5
:102FB00089F0109289020E944F179093B10180937B
:102FC000B0018091B2018823D1F11092B2010E9428
:102FD000441711C08091B201811111C08091B001DC
:102FE0009091B1010E946717069728F081E08093C5
:102FF000B2010E943E178091B201882301F10E9424
:103000003E170E942817882339F1F89421B3939A28
:10301000822F8C6081BB92B38CE0982792BB3FE7F4
:1030200048E391E0315040409040E1F700C000009B
:1030300092B3892782BB21BB9398789408950E940C
:103040009A1980918F02882329F080916D0284FD66
:103050000E94BF0F0C945B18089580914702089559
:1030600008959091B801981307C02091B60130914E
:10307000B70126173707A9F08093B8017093B701FD
:103080006093B6018093B3017093B5016093B4016E
:103090008091A60284FF05C063E083EB91E00C946D
:1030A00096190895BC0184E00C943118BC0183E0AA
:1030B0000C9431180895CF93DF93CAE0D0E080914B
:1030C0006D0284FF18C08091C4019091C5019817CA
:1030D000E1F028E0829FC001112468E08A539E4FEE
:1030E0000E9492198091C40190E001968F709927F7
:1030F0008093C4010AC00E949A198FE99FE001974A
:10310000F1F700C000002197D1F6DF91CF9108952B
:10311000CF93DF93EC01A091C501B0E0CD01019602
:103120008F7099272091C401281779F093E0AA0F96
:10313000BB1F9A95E1F7AA53BE4F98E0FE0101909C
:103140000D929A95E1F78093C5010E949A190E9409
:103150005B1888E0FE01ACEBB1E001900D928A951E
:10316000E1F7DF91CF91089584E690E00895FC01A6
:10317000808180768032A1F58181813061F4848103
:103180009581892B69F58CEB91E090938B0280936C
:103190008A0288E00895823041F486E492E09093B8
:1031A0008B0280938A0281E008958A3021F4838122
:1031B0008093460215C0893099F4828193818115EC
:1031C000924081F484819581892B61F481E0809320
:1031D000BB01868197819093BA018093B90102C0A7
:1031E00080E008958FEF08952091B9013091BA01E0
:1031F000232B71F02091BB01213051F4FC0180811F
:10320000809347021092BA011092B90181E00895AB
:103210008FEF08950895FC0193819330D9F068F4FD
:10322000913081F0923009F059C088E991E0909393
:103230008B0280938A028BE30895913249F1923296
:10324000B9F14CC083ED91E090938B0280938A0298
:1032500082E108958281813099F050F08230F1F559
:1032600085EE91E090938B0280938A028EE0089520
:1032700081E192E090938B0280938A0284E008952A
:1032800085EF91E090938B0280938A028AE1089502
:103290008281882329F0813009F583EC91E002C016
:1032A0008AEA91E090938B0280938A0289E00895E4
:1032B00084819581009751F0019781F485E192E036
:1032C00090938B0280938A0282E3089587E492E0D0
:1032D00090938B0280938A0280E4089580E00895A1
:1032E0001F93CF93DF93162FEA01288124FF05C097
:1032F000398128E82327298302C02AE52883212F42
:10330000FC01CE010296DC0131913D932150121651
:10331000DCF3612F0E9478011C5F1883DF91CF914D
:103320001F9108954DE652E00C94701946EA52E060
:103330000C947019CF93DF9360918C02635067FDFA
:1033400093C080918802CCE0D0E0C81BD109C0575F
:10335000DD4F80918702803120F4CE010E940A194E
:1033600081C08D3209F06EC0683009F07BC083ECFB
:10337000809362028AE580937100109286028881B0
:10338000807621F0CE010E94B71849C09A81109230
:103390006B028981811106C010926C022BE632E02B
:1033A00082E038C0853019F490938D0230C08630A9
:1033B000A1F48B81813041F0823031F0833021F0F3
:1033C000813211F0823221F4CE010E940B1901C02A
:1033D00080E090E49093860222C0883089F08930A2
:1033E00019F490938F0213C08A3069F08B3079F40E
:1033F0008BE480936E028093A70280937A0207C0C9
:103400002FE832E002C02BE632E081E003C02BE679
:1034100032E080E030938B0220938A0209C08F3F14
:1034200039F4988197FD8E8190E89093860207C0C9
:103430009F81911104C09E81981708F4892F809371
:10344000700010C08091860287FF0CC0CE010E94E0
:10345000F4188F3F21F48EE18093710003C0811135
:103460001092700010928C028091710084FF4CC009
:10347000809170008F3F09F447C0C82F893008F051
:10348000C8E08C1B809370009091620288E88927C5
:1034900080936202CC2359F180918A0290918B0231
:1034A0002091860226FF12C0A2E6B2E02C2FAC01CA
:1034B00042565240FA01EA0FFB1FE4911196EC9339
:1034C0001197215011962111F5CF08C0E3E6F2E0E3
:1034D000DC012C2F3D9131932150E1F701962FEF24
:1034E0002C0F820F911D90938B0280938A026C2F78
:1034F00083E692E00E947801CC5FCC3019F08FEF28
:1035000080937000C093710084E190B39C7031F49B
:103510008150D9F710928D0210928502DF91CF91E0
:103520000895CF93DF9385B7886085BF8BB7806898
:103530008BBFCDE6D2E08BE48983A6EAB2E0119698
:103540008C931197E9E7F2E081838AE588838C9375
:103550008083DF91CF91089597FB072E16F4009496
:1035600007D077FD09D00E94C61A07FC05D03EF4AB
:10357000909581959F4F0895709561957F4F08951F
:10358000EE0FFF1F0590F491E02D0994AA1BBB1BC1
:1035900051E107C0AA1FBB1FA617B70710F0A61B53
:1035A000B70B881F991F5A95A9F780959095BC0174
:1035B000CD010895FB01DC0104C08D9101908019BB
:1035C00021F441505040C8F7881B990B0895E199A8
:1035D000FECF9FBB8EBBE09A99278DB30895A8E1DB
:1035E000B0E042E050E00C941A1B262FE199FECF88
:1035F0009FBB8EBBE09A01970DB2021631F02DBB36
:103600000FB6F894E29AE19A0FBE08950396272F19
:103610000E94F61A0E94F51A252F0E94F61A242FEE
:103620000C94F61A0196272F0E94F61A0C94F51A9C
:10363000DC01CB01FC01E199FECF06C0FFBBEEBB74
:10364000E09A31960DB20D9241505040B8F708956E
:04365000F894FFCF1C
:10365400C8007C012D1888185A18561852183018AA
:10366400FF5AE200E900EA00B500B600B700CD0059
:103674008301CC008A0192019401210223022402D5
:103684002502260227022A02B300B4006F0070004C
:10369400818283E200E900EA00B500B600B700CDFC
:1036A400008301CC008A01920194012102230224A7
:1036B400022502260227022A02B300B4006F00701A
:1036C40000818283323336353497969594649363BC
:1036D400926291060531300700FF0100010000FFEE
:0C36E400FF0000010001FF000160006118
:00000001FF
